:020000040000FA
:100000000004040000000000040C0000080C0000C4
:100010000C0C0000100C0000140C0000180C000068
:100020001C0C0000200C0000240C0000280C000018
:100030002C0C0000300C0000340C0000380C0000C8
:100040003C0C0000400C0000440C0000480C000078
:100050004C0C0000500C0000540C0000580C000028
:100060005C0C0000600C0000640C0000680C0000D8
:100070006C0C0000700C0000740C0000780C000088
:100080007C0C0000800C0000840C0000880C000038
:100090008C0C0000900C0000940C0000980C0000E8
:1000A0009C0C0000A00C0000A40C0000A80C000098
:1000B000AC0C0000B00C0000B40C0000B80C000048
:1000C000BC0C0000C00C0000C40C0000C80C0000F8
:1000D000CC0C0000D00C0000D40C0000D80C0000A8
:1000E000DC0C0000E00C0000E40C0000E80C000058
:1000F000EC0C0000F00C0000F40C0000F80C000008
:10010000FC0C0000000D0000040D0000080D0000B4
:100110000C0D0000100D0000140D0000180D000063
:100120001C0D0000200D0000240D0000280D000013
:100130002C0D0000300D0000340D0000380D0000C3
:100140003C0D0000400D0000440D0000480D000073
:100150004C0D0000500D0000540D0000580D000023
:100160005C0D0000600D0000640D0000680D0000D3
:100170006C0D0000700D0000740D0000780D000083
:100180007C0D0000800D0000840D0000880D000033
:100190008C0D0000900D0000940D0000980D0000E3
:1001A0009C0D0000A00D0000A40D0000A80D000093
:1001B000AC0D0000B00D0000B40D0000B80D000043
:1001C000BC0D0000C00D0000C40D0000C80D0000F3
:1001D000CC0D0000D00D0000D40D0000D80D0000A3
:1001E000DC0D0000E00D0000E40D0000E80D000053
:1001F000EC0D0000F00D0000F40D0000F80D000003
:10020000FFFFFF00FFFFFF00040E0000080E0000CC
:100210000C0E0000100E0000140E0000180E00005E
:100220001C0E0000200E0000240E0000280E00000E
:100230002C0E0000300E0000340E0000380E0000BE
:100240003C0E0000400E0000440E0000480E00006E
:100250004C0E0000500E0000540E0000580E00001E
:100260005C0E0000600E0000640E0000680E0000CE
:100270006C0E0000700E0000740E0000780E00007E
:100280007C0E0000800E0000840E0000880E00002E
:100290008C0E0000900E0000940E0000980E0000DE
:1002A0009C0E0000A00E0000A40E0000A80E00008E
:1002B000AC0E0000B00E0000B40E0000B80E00003E
:1002C000BC0E0000C00E0000C40E0000C80E0000EE
:1002D000CC0E0000D00E0000D40E0000D80E00009E
:1002E000DC0E0000E00E0000E40E0000E80E00004E
:1002F000EC0E0000F00E0000F40E0000F80E0000FE
:10030000FC0E0000000F0000040F0000080F0000AA
:100310000C0F0000100F0000140F0000180F000059
:100320001C0F0000200F0000240F0000280F000009
:100330002C0F0000300F0000340F0000380F0000B9
:100340003C0F0000400F0000440F0000480F000069
:100350004C0F0000500F0000540F0000580F000019
:100360005C0F0000600F0000640F0000680F0000C9
:100370006C0F0000700F0000740F0000780F000079
:100380007C0F0000800F0000840F0000880F000029
:100390008C0F0000900F0000940F0000980F0000D9
:1003A0009C0F0000A00F0000A40F0000A80F000089
:1003B000AC0F0000B00F0000B40F0000B80F000039
:1003C000BC0F0000C00F0000C40F0000C80F0000E9
:1003D000CC0F0000D00F0000D40F0000D80F000099
:1003E000DC0F0000E00F0000E40F0000E80F000049
:1003F000EC0F0000F00F0000F40F0000F80F0000F9
:100800000F912000007F24000001880000000000FC
:100810000C000700408B20000100200011000700A1
:10082000000020000000E000020032000000020092
:1008300000000000E2070200000000000040DA00B3
:100840000000FE004440A900000020000000E0007D
:100850000300320000002000A00188004440A800EE
:100860000000060091018800800078000000EB0085
:1008700015003700E280400032A0B4009101BA00B8
:10088000E280400032A0B4009102BA00E280400051
:1008900032A0B4000002EB00472BDE00F507B200E7
:1008A000602CE10004003A000059EB008301E900EC
:1008B000FDFF3E00040037006128E1000100320026
:1008C0000082EB00040007001101BA000200E00002
:1008D000E8FF3A00000006003159BA008301E90040
:1008E0000C0032002159BA008301E90008003200EF
:1008F0000400E00003003A00E280400032A0B400AF
:10090000F5FF370011D9BA008301E900FAFF3A0078
:100910008100E800E180400032A0B4000000060041
:10092000000000000000E00002003200EC62A800BD
:1009300001003700EC62A900000000000000060082
:1009400000000000ECC2BF004300DE006100600058
:10095000000006000001EB0082007800E3FF2100A8
:1009600054C5B30010003700101180006E00600005
:1009700002003200301180002222A90022C2BF00F2
:100980000008A3000800320030118000844F50009E
:1009900008003A000201E800E30F510001003400B2
:1009A000100005008000EB008100E800838F5000FC
:1009B000EDFF34000000050040A7A900A4C6BF0059
:1009C00001CCB300014060005041B300A4E6B70081
:1009D000DAC6BF00014060003040B300DAE6B7007D
:1009E00000000000E0A2A90000000000E0C2A90091
:1009F00000000000E0E2A90000000000F102A900F0
:100A000000000000C862A90000000000C842A90060
:100A100000000000D862A90000000000D882A900F0
:100A200000000000DC62A90000000000C902A9006B
:100A300000000000C922A90000000000C942A9006E
:100A400000000000C962A90000000000C982A900DE
:100A500000000000C9A2A90000000000C9C2A9004E
:100A600000000000C9E2A90000000000E862A9003F
:100A700000000000B00020004011880021E2A80022
:100A800020A2A9002062A800503FB00010118800E9
:100A90008560A9008580A9009560A9009580A900BE
:100AA000000006008040780023C2BF000018A300A9
:100AB000FDFF3A000180FB002011880000000600C5
:100AC000889FBE008A9FBE008C1F780000047800BB
:100AD00050C5B300F3FF070050C5B300F1FF070096
:100AE0000800E00002003A000840780014003700D7
:100AF0000045EB00098020005CC5B3008905440077
:100B000019447800084545008C4F54000400320019
:100B1000E44F540002003200E54F540002003A0056
:100B200050C0B300DFFF070008407800DDFF07007A
:100B30008904E8008B8F5400F1FF3A000A407800E6
:100B40000044EA0050C5B300804F54000400320056
:100B5000E44F540002003200E54F540002003A0016
:100B600050C0B300CFFF070008407800CDFF07005A
:100B700040C0B300CBFF070023C2BF000008A300A2
:100B8000FDFF32004F0678004F05BE004F04BE0047
:100B90000000060080007800101180006E006000E8
:100BA00002003200301180002222A90022C2BF00C0
:100BB0000008A300F8FF3200301180008048780060
:100BC000000006000200FA00889FBE008A1F78001D
:100BD0005AC5B30068805700EEFF07000FF8970072
:100BE0008A4F5000FBFF3A0068805700E9FF07007A
:100BF0000FF897008A4F5000F6FF3A0016003700B2
:100C000068805700E3FF07000FF89700E54F50009A
:100C1000080032008A4F50000F003200E44F5000AD
:100C200006003A00000000000904E000E9FF3A0075
:100C30000C00370068805700D6FF07000FF89700B8
:100C400080C44400005C780070902000800F540045
:100C5000E0FF3200EAFF37008044EB00088020000C
:100C6000E7FF37004F0578004F04BE000080FA0010
:100C700000000600889FBE008A9FBE008C1F78007F
:100C80000204BE004206DD00110032008005EB00C8
:100C90005A80200088007800090078001A010700B7
:100CA000004D78004801DE0012459800214598006B
:100CB0004808DE0030459800E485450062044400A1
:100CC000E0844C00640545008C8F5500F1FF39002D
:100CD0004F0678004F05BE004F04BE00000006001E
:100CE000889FBE008A9FBE008C9FBE008E1F78002A
:100CF0006044B8000202BE004807DD002E0032004A
:100D00008006EB005C8020001C80FB0001F02F00BF
:100D100001046400000474001C4090004800DD00E1
:100D2000F10F200001046400000474002C409000C6
:100D30000080FB0001F02F00818464008084740037
:100D40003C4090004800DD00F10F200081846400E9
:100D500080847400E48646000405BE0000402F0035
:100D6000F1FF2F00040040008580480092BF24005E
:100D700013002000820F5000838F580005003E00B2
:100D80008801780009017800840078000500780067
:100D9000D90007000D04E00002003A001000240012
:100DA000C800070062024500E0824D00640646006C
:100DB0008E8F5600D4FF39004F0778004F06BE00D3
:100DC0004F05BE004F04BE0000000600889FBE0015
:100DD0008A9FBE008C9FBE00800578000202BE0084
:100DE0000000E000160032000005EB000C4020007F
:100DF0000D0020000A05E8000404BE0002402F0098
:100E0000F3FF2F00040041008580490092BF2400B9
:100E100013002000820F5000838F580004003E0012
:100E2000220424008400780005007800BD0007003B
:100E30000802460089824E008A8F5500EDFF3A0075
:100E40004F06BE004F05BE004F04BE000000060066
:100E5000889FBE008A9FBE0008802000184478004A
:100E600019802000994478000904E00005003A0048
:100E700021E2A9000000EB00A9FE07006048800005
:100E8000A600070002C8BF0008E9B70003C8BF00FA
:100E900009E9B70004C8BF000AE9B7000B69EF0011
:100EA000E24F54001C00320005003E000804E00040
:100EB0000A003200E14F54003F003A000D003700B5
:100EC000E64F540038003200E84F5400330032003F
:100ED000E34F540038003A00160037000268EF0074
:100EE00010C0B30003E8B70040002000304888007D
:100EF000310037000984FB004248800053488000DD
:100F0000080078005BFF07004244DD0065044400F0
:100F100038488800280037000980FB0042488000DC
:100F2000534880006EFF0700100020003048880002
:100F3000210037000980FB004248800053488000B0
:100F4000A2FF070010002000304888001A00370078
:100F50000004EB005B802000414880005048800086
:100F60006900070000F47D000804E80040488000A4
:100F70005148800062004000E080480040488800FE
:100F8000514888008A0F5400F3FF39000980FB00A4
:100F9000650040003048880007003700100020003E
:100FA00030488800040037000985FB000904E00090
:100FB000F6FF3200E6FF37004F05BE004F04BE00CB
:100FC00000000600881F78007BFE0700000021005B
:100FD000404888000A29EF004148800050488000BE
:100FE00049000700A2AA2A000300200002006800AE
:100FF00083806800010070000001EA0000017100B8
:101000004F11DE0010C0B300024150000204A200E4
:101010000284FB0000002200404888000A29EF00FB
:10102000414880005048800037000700F2FF2F0041
:10103000F30F2000820F5000838F580005003A0004
:1010400000402000604888000E29EF000004EB00FB
:101050000300370000002200604888000E29EF00DE
:10106000100020002EFE07003AFE07000000E000FE
:1010700008003200E4C2A800400620000000000082
:101080000000E900FDFF3A0050C5B30085FE0700EF
:10109000060037000800E000040032000000EB000A
:1010A0001FFE0700604880001C000700E4C2A80083
:1010B000C4FE070066FF07003048800080FE07007E
:1010C000FBFF3700003B880050052000303B8800C4
:1010D000A00A2000303B880061E7A8000000000063
:1010E0000000000001C8B30061C7BF0001406000FC
:1010F000FDFF3A0000000600900188008308BB0055
:101100008288BB0000000600900188001101BA002F
:101110009181BA000200BE000000060000400100FC
:10112000000006009301800090018800023B8800C7
:101130008108BB0050052000303B8800A00A200039
:10114000303B880061E7A8000000000000000000BC
:1011500001C8B30061C7BF0001406000FDFF3A0055
:101160009301880000000600000800001001000044
:1011700000000000000000000000FE00FFFFFF0074
:10118000FFFFFF00FFFFFF00FFFFFF00FFFFFF006B
:10119000FFFFFF00FFFFFF00FFFFFF00FFFFFF005B
:1011A000FFFFFF00FFFFFF00FFFFFF00FFFFFF004B
:1011B000FFFFFF00FFFFFF00FFFFFF00FFFFFF003B
:1011C000FFFFFF00FFFFFF00FFFFFF00FFFFFF002B
:1011D000FFFFFF00FFFFFF00FFFFFF00FFFFFF001B
:1011E000FFFFFF00FFFFFF00FFFFFF00FFFFFF000B
:1011F000FFFFFF00FFFFFF00FFFFFF00FFFFFF00FB
:020000040002F8
:10AF0000FFFFFF00FFFFFF00FFFFFF00FFFFFF004D
:10AF1000FFFFFF00FFFFFF00FFFFFF00FFFFFF003D
:10AF2000FFFFFF00FFFFFF00FFFFFF00FFFFFF002D
:10AF3000FFFFFF00FFFFFF00FFFFFF00FFFFFF001D
:10AF4000FFFFFF00FFFFFF00FFFFFF00FFFFFF000D
:10AF5000FFFFFF00FFFFFF00FFFFFF00FFFFFF00FD
:10AF6000FFFFFF00FFFFFF00FFFFFF00FFFFFF00ED
:10AF7000FFFFFF00FFFFFF00FFFFFF00FFFFFF00DD
:10AF8000FFFFFF00FFFFFF00FFFFFF00FFFFFF00CD
:10AF9000FFFFFF00FFFFFF00FFFFFF00FFFFFF00BD
:10AFA000FFFFFF00FFFFFF00FFFFFF00FFFFFF00AD
:10AFB000FFFFFF00FFFFFF00FFFFFF00FFFFFF009D
:10AFC000FFFFFF00FFFFFF00FFFFFF00FFFFFF008D
:10AFD000FFFFFF00FFFFFF00FFFFFF00FFFFFF007D
:10AFE000FFFFFF00FFFFFF00FFFFFF00FFFFFF006D
:10AFF000FFFFFF00021E0000BDFA00007F3E0000C0
:00000001FF
